:020000005AC0E4
:0200040012C028
:0200080024C012
:04000C002AC03DC009
:1000120000C0DCB85E9A5E9818955E9AD92C089555
:100022005E9BFBCF9CB808953FB6222019F0922C1C
:100032002224F6DF112019F0912C1124F1DFAA20DD
:1000420019F09A2CAA24ECDF939AF9D03FBE1895A6
:100052003FB654122FC07DBC7CBC44273FBE1895CE
:100062003FB663B7623061F05395523139F45EEFB7
:10007200A52E939872BE54E053BF55273FBE1895E4
:100082003FBE689473BE18953FB60CB14060083FFE
:1000920058F4A0E6B0E0A20FB71D0C9323952936C1
:1000A20009F422273FBE18950E3FE1F3202E9398C4
:1000B2003FBE1895F894E89417E019B9549A579AE4
:1000C200539A8A988E9810E8612E6BBE939A8B9AF7
:1000D20095988D9A919A899A112717BB94988C9A20
:1000E2001FED1DBF22273327772488248394949AF7
:1000F200B3D0959A829BFECF95988299FECF1CB180
:10010200442714E01BBD14E91ABD7DBC7CBC12E47B
:1001120019BF15E01EBD18B7107441F482994AD078
:100122005F9B02C01CB140604330A9F7542E4427A4
:100132001FEF18BF7DBC7CBC15E01EBD80D078943B
:100142000024B82C231711F1E0E6F0E0E30FF71DCD
:100152001081002051F011237AF4703F11F4173FFF
:1001620051F0829B09C000243CC011231AF0082CD4
:10017200172F08C0082C712FF8943395393609F4DB
:100182003327789461D0BB24C82CDCCFE3B7E430AA
:1001920049F0E7EDE2BFE2E0E3BF231739F4EEF7FF
:1001A200E8944DD0C71014C0082C17C073BEE89451
:1001B20046D0CACF959A41608299FECF959808950C
:1001C200112EF8DF1E3F11F4112407C0939805C0C9
:1001D200703F09F4B7CF0024C82C869B6BCF829B5B
:1001E20019C016B3183F60F7002031F011236AF4EA
:1001F200231759F00024A8CF11232AF0142D24D05C
:1002020016B3082C02C0082C412ED4DFB82CCC2403
:100212001BD0E3CFE3B7E43009F409C0E3ECE2BF5B
:10022200E2E0E3BF829907C0EEF7E89408D0B71086
:1002320087CF082C87CF73BEE89401D0D2CF72BE8D
:10024200552714E013BF089573BE5E9BFECF7BBE9D
:100252001CB95E9A6BBE08951BE7FF2706D010E417
:1002620004D017E0F3E701D00895E0EBAE2F08D0F9
:10027200A12F06D0AF2F04D0E395E03CB9F7089543
:100282005D9BFECFACB90000000000005E9AAA2779
:06029200A395F1F70895A9
:00000001FF
